:100000000C9428030C946C030C946C030C946C03F8
:100010000C946C030C946C030C946C030C946C03A4
:100020000C946C030C946C030C946A150C943C16A1
:100030000C949D230C946C030C946C030C946C0333
:100040000C946C030C94CE030C946C030C946C0312
:100050000C946C030C9405240C946C030C946C03AA
:100060000C946C030C946C030C946C030C946C0354
:100070000C946C030C946C030C946C030C946C0344
:100080000C94E30B0C946C030C946C030C946C03B5
:100090000C946C030C946C030C946C030C946C0324
:1000A0000C946C030C946C030C946C03A916CB1683
:1000B000B917CB16B91710173317B91788179B172D
:1000C000851A851AB41AB41AF31A131B691C691C11
:1000D0001E1B691CCE1BCE1B351C3E1C691C631CE1
:1000E000DB1BDB1BDB1BDB1BDB1BDB1BDB1BDB1B60
:1000F000DB1BDB1BDB1BDB1BDB1BDB1BDB1BDB1B50
:10010000EB1BF91B001C071C111C07634236B79B35
:10011000D8A71A39685618AEBAAB558C1D3CB7CC67
:100120005763BD6DEDFD753EF6177231BF000000DF
:10013000803F08000000BE922449123EABAAAA2AC2
:10014000BECDCCCC4C3E00000080BEABAAAAAA3EDD
:1001500000000000BF000000803F00000000000819
:100160004178D3BB4387D1133D190E3CC3BD4282B6
:10017000AD2B3E68EC8276BED98FE1A93E4C80EF74
:10018000FFBE01C4FF7F3F00000000000000000030
:1001900000000000000000010204060A0F17202CD6
:1001A0003A4A5D71879DB3C7DAE9F5FCFFFCF5E9D2
:1001B000DAC7B39D87715D4A3A2C20170F0A0604EF
:1001C0000201000000000000000000000000F1A299
:1001D000F1A32CA4228A3921290014001A00090055
:1001E00013000A000D000F0018001D003602380031
:1001F0002A00040015001600170007000B0011006C
:1002000008000C001200310200301C001B00060028
:10021000190005000E0010003600370024022800E7
:10022000E000E3002B00E200022003200320012075
:100230005000510052004F00010001000100010078
:100240000100010001000100010001003700010070
:100250000100010001000100010001000100010096
:100260000100010001001F02010001000100010066
:100270000100010001000100013064022D020100B3
:100280000100010001000100010001000100010066
:100290000100010001000100000034020000000024
:1002A00000000000000000002F02330200000420C4
:1002B0004C00340000002D00000000000000000091
:1002C0002F00330000004514000000000000000073
:1002D0000000000000000000AD00AC00AB004414C2
:1002E0000100010001000100010001000100010006
:1002F000A800AA00A900AE0030141E021414310098
:10030000210222023500230230022502260230009B
:100310002E021E001F0020002100220023002400C6
:1003200025002600270027020000000000006414BA
:100330002514261424142714081400002D14280052
:1003400001000100010001000100010001000100A5
:100350004A004E004B004D00680069006A006B00C7
:100360006C006D006E006F00700071007200730011
:100370003A003B003C003D003E003F004000410091
:10038000420043004400450000000000000000005F
:100390000000560057000000000000000070000040
:1003A000000031702F703070022001000100010048
:1003B000A800AA00A900AE000651290014001A00E6
:1003C0000800150017001D0018000C001200042082
:1003D00028002A0004001600070009000A000B008C
:1003E0000D000E000F003602E000E1001C001B00B3
:1003F0000600190005001100100037005200240209
:10040000000000002B00E20000002C002C002C015A
:10041000E300500051004F000100000014001A00DA
:10042000090013000A000D005F0060006100000079
:100430002A000000040015001600170007000B003A
:100440005C005D005E004D00E000E1001C001B0050
:100450000600190005000E0059005A005B004E000E
:10046000000000002B00E20000002C002C002C01FA
:100470000000620063005800280354006800650013
:10048000200050006C0061006E0063006B002000D3
:100490004B006500790062006F006100720064002B
:1004A00000002C034F007200740068006F006C00A5
:1004B00069006E0065006100720020004B0065005D
:1004C000790062006F006100720064007300000038
:1004D0000403090409026D00040100A0FA090400E4
:1004E0000001030101000921110100012240000760
:1004F00005810308000A0904010001030102000943
:100500002111010001224D000705820308000A099C
:10051000040200010300000009211101000122363C
:10052000000705830308000A090403000103000013
:100530000009211101000122390007058403100080
:10054000011201100100000008EDFE6060010001D1
:1005500002000105010906A101050719E029E715B7
:1005600000250195087501810205081901290595E5
:10057000057501910295017503910105071900297F
:100580007715002501957875018102C00501098064
:10059000A101850216010026B7001A01002AB70042
:1005A000751095018100C0050C0901A10185031694
:1005B0000100269C021A01002A9C027510950181F7
:1005C00000C005010902A1010901A10005091901E5
:1005D0002905150025019505750181029501750311
:1005E00081010501093009311581257F95027508C2
:1005F000810609381581257F950175088106050C4E
:100600000A38021581257F950175088106C0C0054D
:10061000010906A101050719E029E7150025019543
:1006200008750181029501750881010508190129E4
:10063000059505750191029501750391010507194D
:100640000029FF150026FF00950675088100C000EF
:1006500011241FBECFEFDAE0DEBFCDBF04B603FE2C
:1006600024C080911F0390912003A0912103B09199
:1006700022038730904BA740B04BB9F410921F0370
:1006800010922003109221031092220314BE84B70B
:10069000877F84BF88E10FB6F89480936000109242
:1006A00060000FBEE0E0F8E3099511E0A0E0B1E0E2
:1006B000EEEAFBE502C005900D92A03CB107D9F728
:1006C00013E0A0ECB1E001C01D92AF31B107E1F73A
:1006D0000E94B4120C94D52D0C9400000895089536
:1006E00081E0089508950C946F030C9470030C94AA
:1006F00072030E949F2923E030E0281B3109220F5A
:100700002093C4010895282F2F98809180002111F3
:1007100008C0877F8093800010928D0010928C001B
:100720001BC0886080938000233019F48FEF9FEF07
:100730000FC083E090E0821B9109880F991F2FEF73
:100740003FEFA90102C0569547958A95E2F7CA0185
:1007500090938D0080938C000C9479030E94790310
:1007600084E08093C3011092C0010895279A2F98C6
:100770008FEF9FEF90938700809386008AE08093AD
:10078000800089E1809381000E9408290C94AE03C7
:100790000E94B6036E9A769A0C946E031F920F9283
:1007A0000FB60F9211242F933F938F939F93EF9344
:1007B000FF93E091C101F091C201CF0101969093A6
:1007C000C2018093C1010090C30102C0F695E79574
:1007D0000A94E2F7EF738091C001823019F4E0329D
:1007E00051F404C0813039F4EF3329F480916F0063
:1007F0008D7F80936F00F0E0E457FE4FE49121E09D
:1008000031E0E29FC001E39F900D11240090C401EC
:1008100002C0969587950A94E2F790938D00809395
:100820008C00FF91EF919F918F913F912F910F90AD
:100830000FBE0F901F901895662319F0613089F054
:100840001EC0FC018281882339F081EE0E942919A3
:1008500081E00E94112113C081E00E94322181EECB
:100860000CC0FC018281882339F081EE0E94F119CD
:1008700084E60E94291903C084E60E94F11980E0F1
:1008800090E0089581E008950C94420408950C943A
:10089000C80380911502882309F448C08091D101D2
:1008A0009091D201009779F40E94CF239093D201C6
:1008B0008093D1018091D30190E0009771F48091F1
:1008C000D40190E00AC00E94DB2320910001309106
:1008D00001012817390740F329C00197880F991F94
:1008E000880F991FFC01EB52FE4F6081718182815C
:1008F00093810E94490BE091D30184E0E89FF001CD
:100900001124EB52FE4F60817181828193814FE00F
:1009100050E00E94010F8091D30190E00196609118
:10092000D40170E00E94852D8093D3010C94730351
:10093000109217020C94160B0895089581E080938D
:1009400017020C949D04089508958F929F92AF9280
:10095000BF92EF92FF920F931F93CF93DF93CDB788
:10096000DEB7A3970FB6F894DEBF0FBECDBF7C01F4
:10097000FC0100811181C8010E94CD21B8010E94B3
:1009800039098C01B7010E944404882309F4BDC2CF
:100990000531F0E71F0741F4F7018281882309F44C
:1009A00058C00E94650FB1C20631F0E71F0741F43D
:1009B000F7018281882309F44CC00E946E0FA5C202
:1009C0000731F0E71F0751F4F7018281882309F40A
:1009D00040C00E94610F8111F0CFE3CF0831F0E7F2
:1009E0001F0739F4F7018281882399F10E949E0440
:1009F0008CC20931F0E71F0739F4F701828188239F
:100A000041F10E94980481C20A31F0E71F0749F4BE
:100A1000F70182818823E9F0809117028111F1CFDB
:100A2000E5CF0B31F0E71F0739F4F7018281882306
:100A300081F00E94750F0AC00C31F0E71F0749F4DE
:100A4000F7018281882329F00E94800F0E94A4046C
:100A50005CC280911702811105C0F701828181116A
:100A6000CFC03AC1003E110579F4F7018281882395
:100A700009F44DC00E94160B81E08093160210927B
:100A800015021092D40141C2023E110559F4F7013A
:100A900082818823E1F10E94160B109216021092B7
:100AA000150233C2033E110591F4F70182818823B8
:100AB00071F10E94160B1092160281E080931502CC
:100AC0001092D3011092D2011092D1011EC20235B0
:100AD000110559F4F7018281882309F416C2809127
:100AE0000001909101010A970DC00135110579F4BB
:100AF000F7018281882309F408C280910001909156
:100B000001010A969093010180930001FEC140917A
:100B1000040183E2EFE1F1E0DE01119601900D9214
:100B20008A95E1F7F701808121E030E02C0F3D1F2D
:100B3000280F311DC9012091020130910301FC01F0
:100B4000E20FF31F6081772767FD7095640F711DB9
:100B5000882777FD8095982F0E94A72A20E030E013
:100B600040E451E40E940C2A4B015C01F701218111
:100B700084E090E0821B9109BC01882777FD809575
:100B8000982F0E94A72A9B01AC01C501B4010E94C5
:100B9000A4299B01AC0160E070E080E090E40E9439
:100BA0001A2C20E030E04CED50E40E94B72B4B01B2
:100BB0005C01F70182818823D1F04FE050E0C5014C
:100BC000B4010E94010F809116028823A1F0809148
:100BD000D40124E0829FF0011124EB52FE4F808269
:100BE0009182A282B3828F5F8093D40104C0C50139
:100BF000B4010E94490B0F3F110508F02ECF85C1AB
:100C00008091D00181111FC0043130E7130709F032
:100C100080C00E94460481E08093D0010E94CF23CF
:100C20009093CF018093CE011092C7011092C90119
:100C30001092C8011092CB011092CA011092CD01FE
:100C40001092CC0162C18091CE019091CF010E949F
:100C5000DB23883C910570F48091C701E82FF0E018
:100C6000EE0FFF1FE853FE4F118300838F5F8093C9
:100C7000C7014BC1043180E7180768F4023090E7E0
:100C8000190708F050C00115E0E71E0771F00130A8
:100C90001047A1F11CC1033320E7120709F4E8C093
:100CA0000433104709F4FBC012C1F7018281882385
:100CB00009F412C10E94D41C0E94160B0E949C04CD
:100CC000FFEF24E33CE0F15020403040E1F700C06A
:100CD00000000E942A2419C10431F0E71F0708F020
:100CE000C3C0023020E71207F0F4011530E7130704
:100CF00009F4F2C00130104709F0E9C0F701828120
:100D0000882309F4E9C08091F20281608093F202A5
:100D1000FCC00431F0E71F0708F0A6C0023020E74E
:100D2000120708F4ECC0F7018281882309F4D4C0CB
:100D30000E948E24811102C00E946A240E94A12474
:100D400090E090930403809303030230F0E71F07C1
:100D500021F480910303816080C0033020E71207F3
:100D600021F480910303826078C0043030E71307D8
:100D700021F480910303846070C0053080E7180778
:100D800019F48091030327C0063090E7190721F476
:100D900080910303806161C00730E0E71E0721F402
:100DA00080910303806259C00830F0E71F0721F4E7
:100DB00080910303806451C0093020E7120721F4B9
:100DC00080910303806849C00A3030E7130729F493
:100DD000809103038460886040C00B3080E718076F
:100DE00021F4809103038E7F38C00C3090E71907FF
:100DF00021F4809103038D7F30C00D30E0E71E07A2
:100E000021F4809103038B7F28C00E30F0E71F0789
:100E100019F48091030320C00F3020E7120721F45A
:100E2000809103038F7E19C0003130E7130721F44E
:100E3000809103038F7D11C0013180E7180721F4F1
:100E4000809103038F7B09C0809103030231104717
:100E500011F48F7702C08B7F877F8093030380918B
:100E600003030E94A52451C0033390E71907A1F49E
:100E7000F7018281882321F01092C50182E016C01B
